:103C39000FC30FBF0FBB0FB60FB20FAC0FA70FA16A
:103C49000F9B0F950F8E0F870F800F780F700F68DE
:103C59000F5F0F550F4B0F410F360F2B0F1F0F1211
:103C69000F060EF80EEA0EDB0ECC0EBC0EAB0E9A4A
:103C79000E880E750E620E4E0E390E240E0E0DF7BD
:103C89000DDF0DC70DAE0D940D790D5E0D410D249F
:103C99000D070CE80CC90CA90C890C680C460C23FF
:103CA9000C000BDC0BB80B930B6E0B480B210AFABB
:103CB9000AD30AAC0A840A5B0A330A0A09E109B77A
:103CC900098E0965093B091108E808BE0895086CC1
:103CD9000842081907F107C807A0077807500729FC
:103CE900070206DB06B5068F066A0645062105FDAD
:103CF90005DA05B70595057405530532051204F370
:103D090004D404B60498047B045F04430428040D16
:103D190003F303DA03C103A90391037A0363034D90
:103D290003370322030E02F902E602D302C002AEF0
:103D3900029C028B027A026A025A024B023C022D51
:103D4900021F0211020301F601E901DD01D001C5DB
:103D590001B901AE01A30198018E0184017A0171B3
:103D69000168015F0156014D0145013D0135012EF3
:103D79000126011F01180111010B010400FE00F8C1
:103D890000F200EC00E600E100DC00D600D100CC36
:103D990000C800C300BE00BA00B600010C0101044E
:103DA90002011E030A960401320504040600640791
:103DB900010108000009015A0E01010F000112005A
:103DC9006413010114013C1501FA1664FA17FFFF87
:103DD9001D00072000072400022701012F013C30A4
:103DE900010132010335FFFF3603073CFFFF3DFFA9
:103DF900FF180002191E461A00021B00022D32C8C4
:063E09002E0001FAFAFA96
:10004800900786E0FEA3E0FF7457BE0010D39F40E0
:100058000C903DA312001EE493F599801290078638
:10006800E0FEA3E0FF903DA312001EE493F59990F3
:10007800078612000E900786E0FEA3E0FF746C6FFF
:100088004E700375130022900072E0B402087401E8
:10009800900072F0D20C90013AE090002AF09001A2
:1000A8003BE090002BF090013CE090002CF0A20A7D
:1000B800B3401690013AE0700C90013BE070069056
:1000C800013CE060028002C20A90013AE0B4300FBD
:1000D80090013BE0B4470890013CE0643B6002803B
:1000E80004D20B8002C20BE558B40102800302025D
:1000F80011900057E0F566900062E0F568900063A3
:10010800E0F569900074E0F56A90007AE0900029C3
:10011800F090007CE0F56590007DE0F56790008048
:10012800E0F564900081E0F563900090E090004174
:10013800F0900091E0900042F0900092E09000432F
:10014800F0900093E0900044F0900094E090004517
:10015800F0900095E0900046F0900096E0900047FF
:10016800F0900097E0900048F0900099E0900033FC
:10017800F090009AE0900034F090009BE0900035F9
:10018800F090009CE0900036F0900079E0B4011700
:1001980090000A740FF0A374FFF090000CE4F0A331
:1001A800F07402900079F0900079E0B4035990005F
:1001B8000CE0FEA3E0FF90000AE0FCA3E0FD1200C3
:1001C800037410123F6F7408123F61EF900026F01D
:1001D800EF700674FF900026F07400900079F0909C
:1001E800000BE0900027F090000AE0900028F090C3
:1001F8000026E0900789F0900027E090078AF090A9
:100208000028E090078BF0803F900081E070067531
:100218005801756300A20AB3402E90013AE090009D
:100228002AF090013BE090002BF090013CE0900018
:100238002CF090002AE0700C90002BE070069000E3
:100248002CE060028002C20AE5667003756602E56A
:100258006870037568027E837FC2E5668E048F0529
:10026800FF123F518C398D3AE56975F0FAA4FFAE5B
:10027800F0E5688E048F05FF123F518C3D8D3E904E
:10028800004FE0F56090004DE0FE900069E0B50693
:100298001890004CE0FE900068E0B5060C90004B0A
:1002A800E0FE900059E06E606F900069E070069083
:1002B8000068E060067400900059F0900069E0B4AE
:1002C80002089000497401F08005900049E4F0901C
:1002D8000068E0B4020890004A7401F080059000BC
:1002E8004AE4F0900068E0600690004AE06002800E
:1002F800057560038003756004E559B55802D20C92
:10030800900068E090004CF0900069E090004DF09B
:10031800900059E090004BF0740090009EF074013A
:1003280090009FF074019000A0F074019000A1F07B
:1003380074009000A2F074009000A3F07400900084
:10034800A4F074009000A5F074019000A6F0740069
:100358009000A7F074019000A8F074009000A9F034
:1003680074009000AAF074009000ABF07400900044
:10037800ACF074019000ADF074019000AEF074011F
:100388009000AFF074009000B0F074009000B1F0ED
:1003980074009000B2F07400900362F0740190034E
:1003A80063F07401900364F07401900365F07400C5
:1003B800900366F07400900367F07400900368F08F
:1003C80074009003A2F074019003A3F074019003E9
:1003D800A4F074009003A5F074009003A6F07400D4
:1003E8009003A7F074009003A8F074009003E2F063
:1003F80074009003E3F074019003E4F07401900337
:10040800E5F074009003E6F074009003E7F07400E0
:100418009003E8F07401900422F07400900423F033
:100428007401900424F07400900425F07400900482
:1004380026F07400900427F07400900428F022E558
:10044800B554F7F5B5E5B554FDF5B5C2A2C2A1C2DC
:1004580092C207E5B554FBF5B5755104E55104F5AD
:100468005290004FE0F560900025E4F0C209E5B530
:1004780054FEF5B5C28E758D00758B00754C0075F0
:100488002600752500D28E22750A00750900AE096E
:10049800AF0A7457BE00039F500302054D903DA359
:1004A80012001EE49390004E123F870FBF00010E0A
:1004B800E0FC903DA312001EECFEE493FFEEC39F08
:1004C8005026AE09AF0A0FBF00010E903DA31200DF
:1004D8001EAE09AF0AE493FC903DA312001EE493FC
:1004E80090004E123F87ECF0AE09AF0A903DA31280
:1004F800001EE49390004E123F87E0FC903DA51249
:10050800001EECFCE493FDECD39D4019903DA51230
:10051800001EE493FC903DA312001EE49390004E4D
:10052800123F87ECF0AE09AF0A74022FFF50010E9C
:100538008E098F0A780A740126F6500418E436F6F4
:10054800400302049622750A00750900AE09AF0A35
:100558007415BE00039F500302061B903DFA12005B
:100568001EE49390004E123F870FBF00010EE0FC7F
:10057800903DFA12001EECFEE493FFEEC39F502656
:10058800AE09AF0A0FBF00010E903DFA12001EAE71
:1005980009AF0AE493FC903DFA12001EE493900020
:1005A8004E123F87ECF0AE09AF0A903DFA12001EDA
:1005B800E49390004E123F87E0FC903DFC12001E31
:1005C800ECFCE493FDECD39D4019903DFC12001E19
:1005D800E493FC903DFA12001EE49390004E123F03
:1005E80087ECF0AE09AF0A740F6F4E7006750A15E6
:1005F800750900AE09AF0A74022FFF50010E8E096B
:100608008F0A780A740126F6500418E436F6400377
:1006180002055422054D22054C22054EC2CF2290D8
:10062800F800E4936406600280FE75840175A700F3
:1006380075FF80900788E4F075C91075A70F75A13C
:10064800C775A70075D90075CEFF75A70F75F1FEA0
:1006580075F2FF75F33775F47875A4BA75A5FF754B
:10066800A60775AE0075AFFF75D48175D5FF75D631
:10067800FF75D7FFC296C295C2A0C297E5B554BF11
:10068800F5B5E5B554DFF5B5E5B554EFF5B5E5B520
:10069800547FF5B5E5B554F7F5B5E5B554FDF5B5B1
:1006A80075A70075A20175A14775F80975BC017594
:1006B800BE0475BD6C75BE0775BDA075BE0875BD59
:1006C8000175BC0075BB1875BC2075BA0875E88043
:1006D80075D11375A70F75E10575E20075C74075EB
:1006E8009700759780740A123F417597C0E5975433
:1006F80020700280F8758F0275A700D2AF75980038
:1007080075A90C75A70F75AB4375ADFB75AC1E7558
:10071800A700758911758E00758C00758A00D2A99D
:10072800D28C758D00758B00D2ABD28E75CD0075CD
:10073800CC0075CA0075CB00D2ADC2CFD2CA7591B4
:10074800047592007593CD75EF0675D94075CF0184
:10075800900786E4F0A3F0751300751400C299D2CF
:100768000AC20D12044774C8F518751700122568D7
:1007780075A70FE5FB90001AF0E5FA90001BF0E56D
:10078800F990001CF075A70090F800E493F50812A2
:10079800269F122BD9900789E0900026F090078AAF
:1007A800E0900027F090078BE0900028F090078CED
:1007B800E0900029F090078DE0F56690078EE0F54F
:1007C8006890078FE0F569900790E0F56A900791C7
:1007D800E0F565900792E0F567900793E0F564907F
:1007E8000794E0F563900795E090002AF09007964B
:1007F800E090002BF0900797E090002CF09007987D
:10080800E0900041F0900799E0900042F090079A3C
:10081800E0900043F090079BE0900044F090079C24
:10082800E0900045F090079DE0900046F090079E0C
:10083800E0900047F090079FE0900048F09007A0F4
:10084800E0900033F09007A1E0900034F09007A208
:10085800E0900035F09007A3E0900036F074009027
:100868000082F090013AE0700C90013BE070069035
:10087800013CE060028004C20A8002D20A90F807B4
:10088800E493900021F0900021E0440A900021F0C8
:10089800900021E054FE900021F07406900012F0C0
:1008A8007402900013F090F802E493900014F0742E
:1008B80003900015F07403900016F0741090001760
:1008C800F07405900018F07405900019F090F80481
:1008D800E49390001DF0740090001EF090F805E479
:1008E8009390001FF090F806E493900020F074FFB6
:1008F800900022F0744A900125F07461900126F06E
:100908007474900127F07463900128F0746F90015B
:1009180029F0742090012AF0744A90012BF0745247
:1009280090012CF0743490012DF0743090012EF069
:10093800743590012FF07445900130F074209001C7
:1009480031F07434900132F07453900133F0900018
:100958007AE0D394014006740090007AF07558014B
:10096800755901740390004CF012008F1204901214
:10097800054E122594E5B554FEF5B5900025E4F032
:10098800900786E4F0A3F0752400752300754800ED
:10099800752A007529007549007532007531007592
:1009A8004A00755400755500755A00755104755202
:1009B8000175343C753300757000756F007571CD25
:1009C80075560075570075430075440075450075E8
:1009D8004600755B00754700754200754100900040
:1009E80006E4F0A3F0900008E4F0A3F0755E00754B
:1009F8005F0090000E74FDF0A374E8F0900023E40B
:100A0800F07464900024F0C200D201C202D20375CF
:100A18004D00756D00C294C293C287C290C291C244
:100A28000C7E017F00900028E0123F6F900027E0C5
:100A38002FFF50010E90000AEEF0A3EFF090002671
:100A4800E0700674FF900026F090000AE0FEA3E034
:100A5800FFEFD394FFEE940F400790000AE4F0A351
:100A6800F07400900071F07400900079F0740090B8
:100A78000082F0740090008DF074009000B4F0E5EE
:100A8800677003756704743A90074EF074FD900719
:100A98004FF09003D4E0900414F0D2B0D2B7D2A7AC
:100AA800D2A6D2B1D2A3C207A2B6B39204A2B3B35C
:100AB8009205D29CD2EC75CF01A298B34005C2989A
:100AC800122F3DE5136006A299B3B340028005C218
:100AD800991234ADE51464016005E514B40402808C
:100AE800D5E54DD39405400CE55AC394C85002058A
:100AF8005A754D00E571C394F0501A786F12003F93
:100B0800AE6FAF70EFD394E8EE94034008057175AB
:100B18007000756F00C28E7E047F00E54C123F6F37
:100B2800E58D75F004A4FDACF0EF2DFDEE3CFCE581
:100B38008B75F04084FF7E00ED2FFFEC3EFE8E2586
:100B48008F26D28EA2B6300401B35003020C91A2B4
:100B5800B6300401B35003020C91A2B640670554A5
:100B6800A20D400575FFA0D20DE5B54401F5B5907D
:100B78000024E4F0E554D3956640487C837DC2AEFA
:100B880025AF26123E0F8E238F24E5482FFF5001F4
:100B98000E7401123F618E238F24852448755401F9
:100BA800C28E758D00758B00754C00D28E7403BE95
:100BB80000039F50069000257401F0E543B4060336
:100BC800754300D204A2B6B35003020C91C204903C
:100BD800006BE060181235EEA200B34008E5B5449A
:100BE80008F5B58006E5B554F7F5B58002C2009062
:100BF800006EE06018123743A202B34008E5B5441E
:100C080002F5B58006E5B554FDF5B58006E5B554A1
:100C1800FDF5B5A207B34004D2878002C2879000D1
:100C280059E06004D2908002C29090004AE0B4017A
:100C380004D2948002C294900049E0B40104D29393
:100C48008002C293A209B34004D2918002C291905B
:100C58000018E0FE900014E0C39E4009900014E0E4
:100C6800D39408400974FB900023F01204479000C5
:100C78001DE0601590001DE0FE900017E06E600911
:100C880074FE900023F0120447C2CA7E017F00E57B
:100C98004E123F6FE5CD2FFF50010E8E278F28D2C1
:100CA800CAE565B4014890000EE0FCA3E0FDEFC37F
:100CB8009DEE9C4039B208E52A45296013A208B385
:100CC8004008E5B54404F5B58006E5B554FBF5B52F
:100CD80090000EE0FEA3E0FF900010E0FCA3E0FD12
:100CE800EF2DFDEE3CFC90000EECF0A3EDF0A2B36E
:100CF800300501B35003020DDFA2B3300501B35034
:100D080003020DDFA2B35003020DD80555A20D4012
:100D18000575FFA0D20DE5B54401F5B5900024E4B2
:100D2800F0E555D395685003020DD67CEA7D60AE98
:100D380027AF28123E0F8E298F2AE569123F6F745C
:100D4800FF8E048F05FF123F518C298D2AE5492D0E
:100D5800FD50010C74018C068D07123F618E298F9E
:100D68002A852A49A209B340157464123F6F90007E
:100D780067E08E048F05FF123F518C298D2A755527
:100D88000190000EE0FEA3E0FFAC27AD281200039F
:100D980090000EEEF0A3EFF0E567FF123F51740AE2
:100DA800FF123F5190007BE08C068D07123F6F7455
:100DB800148E048F05FF123F51900010ECF0A3ED44
:100DC800F0C2CA75CD0075CC00754E00D2CAD205E6
:100DD800A2B3B34002C205900025E0B40107E5566E
:100DE800C3940640030213F3E56D902547F82828BD
:100DF80073900059E0C394024003020F4DE551D3AC
:100E080094015003020F4DE55175F040A4FFAEF078
:100E180090031212001EE0C395455018E55175F075
:100E280040A4FFAEF090031112001EE0F52E752DC0
:100E380000020F4DE55175F040A4FFAEF09003108D
:100E480012001EE0C395454003020EE9E55175F016
:100E580040A4FFAEF090031112001EE55175F0405A
:100E6800A4FFAEF0E0FC90030F12001EECFEE0FFC2
:100E7800EEC39FFEE5518E0475F040A4FFAEF090DE
:100E8800031012001EE0F40425458C0088F0A4FF2E
:100E9800AEF0E5518F048E0575F040A4FFAEF090DA
:100EA800031212001EE55175F040A4FFAEF0E0FAFF
:100EB80090031012001EEAFEE0FFEEC39FFECDCCA9
:100EC800CD8E07123F51E55175F040A4FFAEF0906A
:100ED800030F12001EE02DFD50010C8C2D8D2E806D
:100EE80064E55175F040A4FFAEF090030F12001EA8
:100EF800E55175F040A4FFAEF0E0FC90030E12003F
:100F08001EECFEE0FFEEC39F8545F0A4FFAEF0E5C2
:100F1800518F048E0575F040A4FFAEF090031012B7
:100F2800001EE0FECDCCCD8E07123F51E55175F085
:100F380040A4FFAEF090030E12001EE02DFD5001FC
:100F48000C8C2D8D2E756D010213F3900059E0C3A2
:100F58009402400302110190004FE0D395515003D1
:100F68000210A9E55175F040A4FFAEF090031812E5
:100F7800001EE0C395455018E55175F040A4FFAE3A
:100F8800F090031712001EE0F52C752B000210A933
:100F9800E55175F040A4FFAEF090031612001EE074
:100FA800C395454003021045E55175F040A4FFAED6
:100FB800F090031712001EE55175F040A4FFAEF043
:100FC800E0FC90031512001EECFEE0FFEEC39FFE4E
:100FD800E5518E0475F040A4FFAEF09003161200A0
:100FE8001EE0F40425458C0088F0A4FFAEF0E5511E
:100FF8008F048E0575F040A4FFAEF0900318120020
:101008001EE55175F040A4FFAEF0E0FA9003161209
:10101800001EEAFEE0FFEEC39FFECDCCCD8E071288
:101028003F51E55175F040A4FFAEF0900315120052
:101038001EE02DFD50010C8C2B8D2C8064E5517524
:10104800F040A4FFAEF090031512001EE55175F0B4
:1010580040A4FFAEF0E0FC90031412001EECFEE08A
:10106800FFEEC39F8545F0A4FFAEF0E5518F048ED7
:101078000575F040A4FFAEF090031612001EE0FEC6
:10108800CDCCCD8E07123F51E55175F040A4FFAE8F
:10109800F090031412001EE02DFD50010C8C2B8DD6
:1010A8002CE551B40123E560D39401401CE55604B6
:1010B800D395514014E545C39405500D90035FE066
:1010C800A829B80006952A40028003755102E55107
:1010D800B5602290004FE0D395514019E55175F065
:1010E80040A4FFAEF090031712001EE0A823B8003A
:1010F800069524400280020560756D020213F39084
:101108000059E0B4022AE55175F040A4FFAEF09012
:10111800031712001EE0F52C752B00E55175F04001
:10112800A4FFAEF090030E12001EE0F52E752D0000
:10113800900059E0B4030F900051E0F52C752B0096
:10114800752E00752D00756D030213F3E55175F0CA
:1011580040A4FFAEF090032012001EE0C3955A4051
:1011680003021229900049E07036E551D3940140FA
:1011780029AE23AF24AC2DAD2EEDD39FEC9E401AA3
:10118800E55175F040A4FFAEF090031E12001EE07A
:10119800A829B80005D3952A500280021551803439
:1011A800E551D394024029AE23AF24AC2DAD2EEDEA
:1011B800D39FEC9E401AE55175F040A4FFAEF09025
:1011C800031E12001EE0A829B80005D3952A500274
:1011D80080021551E551B55237E551C3956050303D
:1011E800E55604D395514028AE23AF24AC2BAD2C43
:1011F800EFD39DEE9C4019E55175F040A4FFAEF089
:1012080090031F12001EE0A829B80006952A400284
:1012180080020551C292E55165526005C207755AB0
:1012280000756D040213F3E55175F040A4FFAEF0AC
:1012380090031A12001EE0B40117E55175F040A49E
:10124800FFAEF090032012001EE0240AC3955A4016
:10125800030212FF753064752F00A207B3500B907C
:101268000060E02405C3954540030212FFE551756F
:10127800F040A4FFAEF090031D12001EE0C3954598
:101288004064E55175F040A4FFAEF090031C1200D5
:101298001EE55175F040A4FFAEF0E0FC90031B1270
:1012A800001EECFEE0FFEEC39F8545F0A4FFAEF004
:1012B800E5518F048E0575F040A4FFAEF090031D34
:1012C80012001EE0FECDCCCD8E07123F51E55175C0
:1012D800F040A4FFAEF090031B12001EE02DFD505D
:1012E800010C8C2F8D30AE23AF24AC2FAD30EFD353
:1012F8009DEE9C4002D207756D050213F3E551B4CB
:101308000109900059E0C3940240030213D39003EB
:1013180058E0D3954550030213D3900356E0C39584
:10132800455040900357E0FE900355E0F4042EFE2C
:10133800900356E0F40425458E0088F0A4FFAEF033
:10134800900358E0FC900356E0F4042C8E048F05BB
:10135800FF123F51900355E02DFD50010C8C2B8D51
:101368002C802C900355E0FE900354E0F4042E8565
:1013780045F0A4FFAEF0900356E08E048F05FF12EF
:101388003F51900354E02DFD50010C8C2B8D2CE522
:1013980051C395605030E55604D395514028AE238B
:1013A800AF24AC2BAD2CEFD39DEE9C4019E55175C5
:1013B800F040A4FFAEF090031F12001EE0A829B869
:1013C8000006952A40028003755102900049E0B456
:1013D8000106E551640160028003755102E551651B
:0B13E800526005C207755A00756D00C9
:10254700020DF9020F5302110702115402122F0252
:0225570013056A
:1013F300900050E02402A823B80007D395244002AC
:10140300C207900025E0B40109900059E0C394039A
:10141300400302157B900049E060030214CAE551C2
:10142300D394014034E55175F040A4FFAEF090032E
:101433001412001EE0A823B8001FD39524401AE518
:101443005175F040A4FFAEF090031F12001EE0A8F8
:1014530029B80005D3952A500280021551E551D3CE
:101463009401402FE55175F040A4FFAEF0900312B4
:1014730012001EE0C39545501AE55175F040A4FFD4
:10148300AEF090031E12001EE0A829B80005D39504
:101493002A500280021551E551D394014022E556AA
:1014A30004C39551501AE55175F040A4FFAEF09076
:1014B300031E12001EE0A829B80005D3952A500286
:1014C30080021551021570E551D394024034E55161
:1014D30075F040A4FFAEF090031412001EE0A823A1
:1014E300B8001FD39524401AE55175F040A4FFAE10
:1014F300F090031F12001EE0A829B80005D3952A17
:10150300500280021551E551D39402402FE55175E5
:10151300F040A4FFAEF090031212001EE0C3954505
:10152300501AE55175F040A4FFAEF090031E12006F
:101533001EE0A829B80005D3952A50028002155150
:10154300E551D394024022E55604C39551501AE560
:101553005175F040A4FFAEF090031E12001EE0A8E8
:1015630029B80005D3952A500280021551E551652B
:10157300526005C207755A00900060E0D39545504C
:1015830009900054E0C395455002C207900059E00A
:1015930070030217E0A2A5B34008A2A4B34003025C
:1015A30017C9AE35AF367441D39F749C9E400578FE
:1015B3003512003FAE35AF36EFB48806EEB41302F2
:1015C30080030217A6A2A55003021669900059E0F2
:1015D300B4010B90004FE0D395604002056090008A
:1015E30059E0B40254E55175F040A4FFAEF0900306
:1015F3002012001EE0C3955A503F90004FE0D39550
:10160300514021E55604D395514019E55175F040F9
:10161300A4FFAEF090031412001EE0A823B8000646
:10162300952440028002055190004FE0F560E5519A
:1016330065526005C207755A00900059E0B403264D
:1016430090004FE0D395514008E55604D39551508F
:10165300028002055190004FE0F560E5516552604C
:1016630005C207755A00A2A450030217A690005999
:10167300E0B4016E900049E07035E551D394014028
:1016830029E55175F040A4FFAEF090031E12001E31
:10169300E0A829B8000FD3952A400A1551755A00BE
:1016A300855160800385516080037560018033E557
:1016B30051D394024029E55175F040A4FFAEF09058
:1016C300031E12001EE0A829B8000FD3952A400A72
:1016D3001551755A008551608003855160800375EB
:1016E3006002900059E0D39401500302179AE55128
:1016F30075F040A4FFAEF090032012001EE0C395E6
:101703005A400302179A900049E07041E551D3947F
:10171300014034E55175F040A4FFAEF0900311127F
:10172300001EE0A823B8001FD39524401AE5517585
:10173300F040A4FFAEF090031E12001EE0A829B8EB
:101743000005D3952A500280021551803FE551D3FD
:1017530094024034E55175F040A4FFAEF0900311BC
:1017630012001EE0A823B8001FD39524401AE551A8
:1017730075F040A4FFAEF090031E12001EE0A829EE
:10178300B80005D3952A500280021551E5516552E0
:101793006005C207755A00E556B40704055E800369
:1017A300755E00E563B4010EAE35AF36EF6440708D
:1017B30005EE649C6002800EA2A54003755801A249
:1017C300A44003755802A2A5B3B35006A2A4B3B3B1
:1017D300400280067536007535000218CEA2A5B307
:1017E3004008A2A4B340030218BAAE35AF36744121
:1017F300D39F749C9E4005783512003FAE35AF36BB
:10180300EFB48806EEB4130280030218BAA2A5400F
:101813006F900068E0605A90004AE0B401079000BE
:101823004AE4F0800690004A7401F090004AE070A8
:1018330005756003800375600490004AE0B40104F9
:10184300D2948002C294E551B4041AE55175F04074
:10185300A4FFAEF090031E12001EE0A829B80005F5
:10186300D3952A50028008755103C207755A008028
:1018730003756004E556B40704055E8003755E00D6
:10188300A2A44033900069E06021900049E0B401D4
:1018930007900049E4F080069000497401F090003D
:1018A30049E0B40104D2938002C293E556B407041D
:1018B300055E8003755E00A2A5B3B35006A2A4B370
:1018C300B340028006753600753500E558655960EA
:1018D30006900082E06003021A56C29C75140075DC
:1018E3001300C2CAE558902559F8282873801212AC
:1018F3002BD9800D122CB28008122D8B8003122E4F
:01190300647F
:0F2559000218F00218F20218F70218FC0219011A
:10190400900029E090007AF0E566900057F0E568D1
:10191400900062F0E569900063F0E56A900074F06D
:10192400E56590007CF0E56790007DF0E56490004B
:1019340080F0E563900081F090002AE090013AF095
:1019440090002BE090013BF090002CE090013CF0E3
:10195400900041E0900090F0900042E0900091F0FF
:10196400900043E0900092F0900044E0900093F0E7
:10197400900045E0900094F0900046E0900095F0CF
:10198400900047E0900096F0900048E0900097F0B7
:10199400900033E0900099F0900034E090009AF0C9
:1019A400900035E090009BF0900036E090009CF0B1
:1019B4007400900082F0744A900125F074619001E3
:1019C40026F07474900127F07463900128F0746F0A
:1019D400900129F0742090012AF0744A90012BF0B0
:1019E400745290012CF0743490012DF074309001F5
:1019F4002EF0743590012FF07445900130F074206E
:101A0400900131F07434900132F07453900133F04A
:101A14009003D4E0900414F0743A90074EF074FDEF
:101A240090074FF012008F900004E4F0A3F09000B0
:101A3400067475F0A37430F09000087475F0A37404
:101A440030F0855859D2CA754C00D29C741B900052
:101A540023F0E556C394065005E551B55203021A26
:101A6400F6C207E55175F040A4FFAEF090032212D0
:101A7400001EE030E003D38001C39296E55175F077
:101A840040A4FFAEF090032312001EE030E003D325
:101A94008001C39295E556B40106E55164016002E4
:101AA4008004C2A08019E55175F040A4FFAEF09007
:101AB400032412001EE030E003D38001C392A0E5AA
:101AC4005175F040A4FFAEF090032512001EE030E3
:101AD400E003D38001C39297855152AE29AF2A7493
:101AE40005BE00039F5007E545D3940550028002CC
:101AF400D292E556D394055003021C43C207E55124
:101B0400D394015003021B98E55175F040A4FFAE35
:101B1400F090031E12001EE0A829B80007D3952AEE
:101B240040021551E55165526067E55175F040A4D6
:101B3400FFAEF090032212001EE030E003D38001D8
:101B4400C39296E55175F040A4FFAEF090032312C2
:101B5400001EE030E003D38001C39295E55175F097
:101B640040A4FFAEF090032412001EE030E003D343
:101B74008001C392A0E55175F040A4FFAEF090033C
:101B84002512001EE030E003D38001C392978551F3
:101B940052021C43E556B406349000ACE030E00336
:101BA400D38001C392969000ADE030E003D380016E
:101BB400C392959000AEE030E003D38001C392A0BD
:101BC4009000AFE030E003D38001C39297E556B4B0
:101BD40007349000A5E030E003D38001C3929690CF
:101BE40000A6E030E003D38001C392959000A7E003
:101BF40030E003D38001C392A09000A8E030E0035A
:101C0400D38001C39297E556B4083490009EE03027
:101C1400E003D38001C3929690009FE030E003D3A9
:101C24008001C392959000A0E030E003D38001C30B
:101C340092A09000A1E030E003D38001C39297907A
:101C44000072E06058E54575F00284FF7E00900163
:101C54004E12001EE0F55CE54775F00A84FF7E0035
:101C640090024E12001EE0F55DE55C255DD39464A0
:101C7400400BE55C255DC39464F55C8003755C00F2
:101C8400E55C75F00284FF7E008F5CEFC3943350F3
:101C940007EF24CDF55C8003755CFF801CE545757A
:101CA400F00284FF7E0090014E12001EE075F002E7
:101CB40084FF7E00EF24CDF55CE595C3955C40047C
:101CC400C2A28002D2A2A207B34005E556B407031C
:101CD4007571CDE595C395714004C2A18002D2A16E
:101CE400E543C3940640030222E7A2EDB350030286
:101CF40022E7C2EDE5436003021E497E017F00E551
:101D0400BE123F6FE5BD2FFF50010E900000EEF0B4
:101D1400A3EFF0900029E0B401177E0F7FFF90003D
:101D240000E0FCA3E0FD120003900000EEF0A3EF3E
:101D3400F0900079E0B4025B900000E0FEA3E0FFC5
:101D440090000AE0FCA3E0FDEDD39FEC9E400F90D1
:101D54000000E0F8A3E090000AC8F0A3C8F09000E7
:101D640000E0FEA3E0FF90000CE0FCA3E0FDEFD355
:101D74009DEE9C400F900000E0F8A3E090000CC89A
:101D8400F0A3C8F0900000E0FEA3E0FF7404123F4B
:101D9400618F44900079E07060900000E0FEA3E061
:101DA400FF90000AE0FCA3E0FDEFD39DEE9C400D04
:101DB400120003900000EEF0A3EFF0800790000003
:101DC400E4F0A3F0900000E0FEA3E0FF7410123FE3
:101DD4006F900026E08E048F05FF123F51900000A3
:101DE400ECF0A3EDF07400D39D74019C40089000C6
:101DF40001E0F54480037544FFE54475F00AA4FF4F
:101E0400AEF074198E048F05FF123F518D45ED25F8
:101E140032FFAE3150010E7401123F618F4585458A
:101E240032753100EFD394624003754562900072BD
:101E3400E064016006900066E0600280057543017D
:101E4400800375BB17E543B401028003021F397E8A
:101E5400017F00E5BE123F6FE5BD2FFF50010E90DC
:101E64000000EEF0A3EFF0900072E0B4017EE534E0
:101E740045336025AC33AD341DBDFF011C8F028E8C
:101E8400038C068D07903C3912002EE493FE7401F6
:101E940093FFEFC39AEE9B400280057833123F997B
:101EA400AE33AF3474B3BE0025D39F4021900000FD
:101EB400E0FCA3E0FD0FBF00010E903C3912002EA0
:101EC400E493FE740193FFEDC39FEC9E40028005F2
:101ED400783312003FAE33AF34E56A123F6F746457
:101EE4008E048F05FF123F518D478033900066E0CA
:101EF400602D900000E0FEA3E0FFEFD39400EE9489
:101F040008400F900066E0B40104C2098002D209BF
:101F1400800D900066E0B40104D2098002C20990E9
:101F24000072E064026006900066E0600575BB160E
:101F34008003754302E543B4020280030220277E36
:101F4400017F00E5BE123F6FE5BD2FFF50010E90EB
:101F54000000EEF0A3EFF0900072E0B4027EE534EE
:101F640045336025AC33AD341DBDFF011C8F028E9B
:101F7400038C068D07903ACF12002EE493FE740171
:101F840093FFEFC39AEE9B400280057833123F998A
:101F9400AE33AF3474B3BE0025D39F40219000000C
:101FA400E0FCA3E0FD0FBF00010E903ACF12002E1B
:101FB400E493FE740193FFEDC39FEC9E4002800501
:101FC400783312003FAE33AF34E56A123F6F746466
:101FD4008E048F05FF123F518D478033900066E0D9
:101FE400602D900000E0FEA3E0FFEFD39400EE9498
:101FF40008400F900066E0B40104C2098002D209CF
:10200400800D900066E0B40104D2098002C20990F8
:102014000072E07003754700900066E07002C20928
:1020240075BB1FE543B403457E017F00E5BE123F47
:102034006FE5BD2FFF50010E900000EEF0A3EFF00E
:102044007409123F6F74E68E048F05FF123F518CA2
:10205400418D42E54A2DFD50010C74018C068D071B
:10206400123F618E418F4285424A75BB19E543B4E4
:10207400040280030221CF7E017F00E5BE123F6F80
:10208400E5BD2FFF50010E900000EEF0A3EFF074B9
:1020940004123F618F4BE564B40102800302215CAA
:1020A400756B00756B00E56BD394074003022149FF
:1020B400E56B900041123F87E0D3954B501AE56BD6
:1020C400900041123F87E0F404254BFEE56B90003D
:1020D40037123F87EEF08017E56B900041123F877F
:1020E400E0C3954BFEE56B900037123F87EEF0E5B9
:1020F4006BC394044009900084E0C3956B503BE5A6
:102104006B6029E56B900037123F87FEE0FFEE908D
:10211400003FE0D39F4013E56B900037123F87E008
:1021240090003FF0E56B900040F0800E900037E0A7
:1021340090003FF07400900040F0786B740126F634
:1021440040030220AA900040E0F4042408F556E578
:1021540056D394054002C292E564D39401402FE51E
:102164004BD3946E4004D20E8002C20E755605E520
:1021740064B40205A20EB340028003755607E564F9
:10218400B40306A20EB3B340028003755607E557A5
:1021940065566008E55104F552855657E556B4076F
:1021A40008E5B54480F5B58006E5B5547FF5B5E599
:1021B4005664066005E556B40808E5B54410F5B55F
:1021C4008006E5B554EFF5B575BB13E543B40502D8
:1021D40080030222E37E017F00E5BE123F6FE5BD6E
:1021E4002FFF50010E900000EEF0A3EFF0740412E4
:1021F4003F618F46E563B4020280030222E0756BFF
:1022040000756B00E56BD394034003022297E56BE2
:10221400900033123F87E0D39546501AE56B900047
:1022240033123F87E0F4042546FEE56B90002D123F
:102234003F87EEF08017E56B900033123F87E0C3D1
:102244009546FEE56B90002D123F87EEF0E56B603E
:1022540029E56B90002D123F87FEE0FFEE900031E0
:10226400E0D39F4013E56B90002D123F87E0900070
:1022740031F0E56B900032F0800E90002DE090007C
:1022840031F07400900032F0786B740126F640034C
:10229400022208900082E07043E52A45296036E571
:1022A40058C39403500A900032E004C394034002DC
:1022B4008007900032E004F558E558D39402400AB0
:1022C400900032E004D3940250028007900032E080
:1022D40004F5588007900032E004F55875BB1805E2
:1022E40043D2ECE55ED39404500302240175CF017C
:1022F400C2A2AE35AF367488D39F74139E4005A234
:10230400A5B34014AE35AF367488D39F74139E4082
:1023140005A2A4B340028048783512003FAE35AF21
:1023240036EFB4883BEEB41337A2A5B3500990003E
:102334004FE0D395515002800405518011A2A5B3FA
:10234400500890004FE0655160028002D207A2A4B9
:10235400B35007E551D39401500280041551C207CC
:10236400A2A5B3B35006A2A4B3B340028006753647
:1023740000753500E55165526067E55175F040A47C
:10238400FFAEF090032212001EE030E003D3800180
:10239400C39296E55175F040A4FFAEF0900323126A
:1023A400001EE030E003D38001C39295E55175F03F
:1023B40040A4FFAEF090032412001EE030E003D3EB
:1023C4008001C392A0E55175F040A4FFAEF09003E4
:1023D4002512001EE030E003D38001C3929785519B
:1023E40052A20740057571CD80037571FFE595C351
:1023F40095714004C2A18002D2A10222F1A20DB3C0
:10240400500DAE25AF2674E8C39F74039E4002802E
:102414000B75FFA0D20DE5B554FBF5B5AE25AF267F
:10242400EFD39420EE944E500302251B120447C2AE
:102434008E758D00758B00754C00D28EC207757039
:1024440000756F007571CD755104752400752300F6
:10245400755400755A00C287900059E06004D29008
:102464008002C29090004AE0B40104D2948002C277
:1024740094900049E0B40104D2938002C293A2096B
:10248400B34004D2918002C29190006BE0601812B4
:1024940035EEA200B34008E5B54408F5B58006E57D
:1024A400B554F7F5B58002C20090006EE0601812D2
:1024B4003743A202B34008E5B54402F5B58006E50A
:1024C400B554FDF5B58006E5B554FDF5B590000E9F
:1024D40074FDF0A374E8F0E543B40603754300907B
:1024E4000025E4F0752600752500758D00758B00B8
:1024F400754C00900024E0C394035008900024E03D
:1025040004F080067403900024F0900024E0B403E7
:1025140006E5B554FEF5B5AE27AF28EFD39410EE1B
:102524009427401CC2CA75CD0075CC00752800756F
:102534002700D2CA754E00752A007529007555000A
:03254400020ABECA
:1038F50000000100013201640196019602000212E6
:1039050002240200020003000340038003C00400F8
:103915000440048004C005000600060006000600F9
:10392500060006000600060000FF0131016301954F
:1039350001FF01FF0211022302FF02FF02FF033F05
:10394500037F03BF03FF043F047F04BF04FF05FF9C
:1039550006FF06FF06FF06FF06FF06FF06FF06FF3A
:103965000FAA0FA50F9F0F9A0F940F8D0F870F802A
:103975000F780F710F680F600F570F4E0F450F3BF4
:103985000F300F250F1A0F0E0F020EF50EE80EDB86
:103995000ECC0EBE0EAE0E9F0E8E0E7D0E6C0E5A0A
:1039A5000E470E340E200E0C0DF70DE20DCB0DB5A6
:1039B5000D9D0D850D6D0D540D3A0D200D050CE970
:1039C5000CCE0CB10C940C760C580C3A0C1B0BFB62
:1039D5000BDB0BBB0B9A0B790B570B350B130AF152
:1039E5000ACE0AAB0A870A640A400A1C09F809D4F8
:1039F50009B0098C09670943091F08FB08D608B2F5
:103A0500088E086A0846082307FF07DC07B90796EA
:103A150007730751072F070D06EC06CA06AA068984
:103A250006690649062A060A05EC05CD05B0059284
:103A350005750558053C0520050504EA04CF04B5C0
:103A4500049C04820469045104390422040B03F420
:103A550003DE03C803B2039D038903750361034DA8
:103A6500033B03280316030402F202E102D102C05C
:103A750002B002A002910282027302650257024956
:103A8500023C022F02220216020901FD01F201E6A3
:103A950001DB01D001C601BB01B101A7019D019464
:103AA500018B0182017901700168016001580150A3
:103AB5000148014101390132012B0125011E01187F
:103AC5000111010B010500FF00FA0FA60FA00F99C8
:103AD5000F920F8B0F840F7C0F740F6B0F620F58B3
:103AE5000F4E0F430F380F2C0F1F0F120F050EF738
:103AF5000EE80ED80EC80EB70EA50E930E800E6CEE
:103B05000E580E420E2C0E150DFD0DE40DCB0DB10C
:103B15000D950D790D5D0D3F0D200D010CE10CC0CE
:103B25000C9E0C7C0C590C350C100BEA0BC40B9E2F
:103B35000B760B4F0B260AFD0AD40AAA0A800A55F2
:103B45000A2A09FF09D409A8097C0950092508F999
:103B550008CD08A10875084A081E07F307C8079D80
:103B650007730749072006F706CE06A6067E065701
:103B75000630060A05E405BF059B057705540532A1
:103B8500051004EF04CE04AE048F0471045304350C
:103B9500041903FD03E203C703AD0394037B036329
:103BA500034B0334031E030802F302DE02CA02B606
:103BB50002A30291027F026D025C024C023C022CC0
:103BC500021D020E020001F201E401D701CA01BE85
:103BD50001B101A6019A018F0185017A0170016683
:103BE500015D0153014A01410139013101290121D9
:103BF50001190112010B010400FD00F700F000EAB4
:103C050000E400DE00D900D300CE00C900C400BF27
:103C150000BA00B500B100AD00A800A400A0009C4A
:103C2500009900950091008E008A0087008400812C
:043C3500007E007B92
:10256800751A00751900AE19AF1AAC17AD18EDC37E
:102578009FEC9E401674FF123F4175CF01781A7484
:102588000126F6500418E436F650DB22900786E45C
:10259800F0A3F0751000750F00751300751400C2D4
:1025A8000FD21022C2AF75D900758F0375B7A57504
:1025B800B7F190F800E4F0758F0175B7A575B7F11C
:1025C800E50890F800F075B7A575B7F190F801E443
:1025D800F075B7A575B7F190079DE090F802F07512
:1025E800B7A575B7F19007A1E090F803F075B7A506
:1025F80075B7F190079EE090F804F075B7A575B728
:10260800F190079FE090F805F075B7A575B7F190C0
:1026180007A0E090F806F075B7A575B7F19007A286
:10262800E090F807F0758F0075D940D2AF22900777
:1026380088E0B4AB61C2AF75D90075B62275F522D2
:10264800758F0375B7A575B7F1740090F600F0752E
:102658008F01750A00750900AE09AF0A7413BE0030
:10266800279F402475B7A575B7F190078912001EFA
:10267800E0FC90F60012001EECF0780A740126F6D1
:10268800500418E436F650D0758F0075F51175B6FC
:102698002075D940D2AF22C2AF75D90075F5227521
:1026A8000A00750900AE09AF0A7413BE00229F40E4
:1026B8001F90F60012001EE493FC90078912001E7A
:1026C800ECF0780A740126F6500418E436F650D572
:1026D80075F51175D940D2AF22900788E0B4AA02E7
:1026E800800302281EC2AF75D90075B62275F5227F
:1026F800758F0375B7A575B7F1740090EE00F07586
:10270800B7A575B7F1740090F000F075B7A575B767
:10271800F1740090F200F075B7A575B7F1740090E8
:10272800F400F0758F01750A00750900AE09AF0A4B
:1027380074FFC39F74019E402475B7A575B7F190C7
:10274800004E12001EE0FC90EE0012001EECF07825
:102758000A740126F6500418E436F650CF750A00BC
:10276800750900AE09AF0A74FFC39F74019E402427
:1027780075B7A575B7F190024E12001EE0FC90F0F7
:102788000012001EECF0780A740126F6500418E4D2
:1027980036F650CF750A00750900AE09AF0A74FF06
:1027A800C39F74019E402475B7A575B7F190044E78
:1027B80012001EE0FC90F20012001EECF0780A7481
:1027C8000126F6500418E436F650CF750A0075094C
:1027D80000AE09AF0A74FFC39F74019E402475B709
:1027E800A575B7F190064E12001EE0FC90F4001299
:1027F800001EECF0780A740126F6500418E436F648
:1028080050CF758F0075F51175B62075D940D2AFC8
:10281800743A90074EF022900788E0B4AA02800329
:1028280002295CC2AF75D90075B62275F522758F7D
:102838000375B7A575B7F1740090E600F075B7A5F4
:1028480075B7F1740090E800F075B7A575B7F17425
:102858000090EA00F075B7A575B7F1740090EC0028
:10286800F0758F01750A00750900AE09AF0A74FF8B
:10287800C39F74019E402475B7A575B7F190004EAB
:1028880012001EE0FC90E60012001EECF0780A74BC
:102898000126F6500418E436F650CF750A0075097B
:1028A80000AE09AF0A74FFC39F74019E402475B738
:1028B800A575B7F190024E12001EE0FC90E80012D8
:1028C800001EECF0780A740126F6500418E436F677
:1028D80050CF750A00750900AE09AF0A74FFC39F8F
:1028E80074019E402475B7A575B7F190044E120087
:1028F8001EE0FC90EA0012001EECF0780A74012633
:10290800F6500418E436F650CF750A00750900AE83
:1029180009AF0A74FFC39F74019E402475B7A5755B
:10292800B7F190064E12001EE0FC90EC0012001E5B
:10293800ECF0780A740126F6500418E436F650CF05
:10294800758F0075F51175B62075D940D2AF743AF8
:1029580090074EF022900788E0B4AA028003022A6A
:102968009AC2AF75D90075B62275F522758F0375B1
:10297800B7A575B7F1740090DE00F075B7A575B707
:10298800F1740090E000F075B7A575B7F174009088
:10299800E200F075B7A575B7F1740090E400F07522
:1029A8008F01750A00750900AE09AF0A74FFC39F4D
:1029B80074019E402475B7A575B7F190004E1200BA
:1029C8001EE0FC90DE0012001EECF0780A7401266E
:1029D800F6500418E436F650CF750A00750900AEB3
:1029E80009AF0A74FFC39F74019E402475B7A5758B
:1029F800B7F190024E12001EE0FC90E00012001E9B
:102A0800ECF0780A740126F6500418E436F650CF34
:102A1800750A00750900AE09AF0A74FFC39F7401F7
:102A28009E402475B7A575B7F190044E12001EE0BC
:102A3800FC90E20012001EECF0780A740126F650B1
:102A48000418E436F650CF750A00750900AE09AFD0
:102A58000A74FFC39F74019E402475B7A575B7F12A
:102A680090064E12001EE0FC90E40012001EECF0EE
:102A7800780A740126F6500418E436F650CF758F9C
:102A88000075F51175B62075D940D2AF743A900724
:102A98004EF022900788E0B4AA028003022BD8C225
:102AA800AF75D90075B62275F522758F0375B7A570
:102AB80075B7F1740090D600F075B7A575B7F174C5
:102AC8000090D800F075B7A575B7F1740090DA00DA
:102AD800F075B7A575B7F1740090DC00F0758F013B
:102AE800750A00750900AE09AF0A74FFC39F740127
:102AF8009E402475B7A575B7F190004E12001EE0F0
:102B0800FC90D60012001EECF0780A740126F650EC
:102B18000418E436F650CF750A00750900AE09AFFF
:102B28000A74FFC39F74019E402475B7A575B7F159
:102B380090024E12001EE0FC90D80012001EECF02D
:102B4800780A740126F6500418E436F650CF750A50
:102B580000750900AE09AF0A74FFC39F74019E4057
:102B68002475B7A575B7F190044E12001EE0FC90CD
:102B7800DA0012001EECF0780A740126F6500418E8
:102B8800E436F650CF750A00750900AE09AF0A742D
:102B9800FFC39F74019E402475B7A575B7F19006D1
:102BA8004E12001EE0FC90DC0012001EECF0780AC9
:102BB800740126F6500418E436F650CF758F007568
:102BC800F51175B62075D940D2AF743A90074EF01A
:102BD80022C2AF75D90075F522750A00750900AED5
:102BE80009AF0A74FFC39F74019E401F90EE001244
:102BF800001EE493FC90004E12001EECF0780A745C
:102C08000126F6500418E436F650D4750A00750902
:102C180000AE09AF0A74FFC39F74019E401F90F075
:102C28000012001EE493FC90024E12001EECF07895
:102C38000A740126F6500418E436F650D4750A00D2
:102C4800750900AE09AF0A74FFC39F74019E401F47
:102C580090F20012001EE493FC90044E12001EEC49
:102C6800F0780A740126F6500418E436F650D47544
:102C78000A00750900AE09AF0A74FFC39F74019E6C
:102C8800401F90F40012001EE493FC90064E1200C0
:102C98001EECF0780A740126F6500418E436F65053
:102CA800D475F51175D940D2AF22C2AF75D9007568
:102CB800F522750A00750900AE09AF0A74FFC39FB3
:102CC80074019E401F90E60012001EE493FC9000E1
:102CD8004E12001EECF0780A740126F6500418E42F
:102CE80036F650D4750A00750900AE09AF0A74FFAC
:102CF800C39F74019E401F90E80012001EE493FCDD
:102D080090024E12001EECF0780A740126F6500468
:102D180018E436F650D4750A00750900AE09AF0AF2
:102D280074FFC39F74019E401F90EA0012001EE4C6
:102D380093FC90044E12001EECF0780A740126F6FB
:102D4800500418E436F650D4750A00750900AE0927
:102D5800AF0A74FFC39F74019E401F90EC001200DD
:102D68001EE493FC90064E12001EECF0780A7401E3
:102D780026F6500418E436F650D475F51175D94086
:102D8800D2AF22C2AF75D90075F522750A00750950
:102D980000AE09AF0A74FFC39F74019E401F90DE06
:102DA8000012001EE493FC90004E12001EECF07816
:102DB8000A740126F6500418E436F650D4750A0051
:102DC800750900AE09AF0A74FFC39F74019E401FC6
:102DD80090E00012001EE493FC90024E12001EECDC
:102DE800F0780A740126F6500418E436F650D475C3
:102DF8000A00750900AE09AF0A74FFC39F74019EEB
:102E0800401F90E20012001EE493FC90044E120052
:102E18001EECF0780A740126F6500418E436F650D1
:102E2800D4750A00750900AE09AF0A74FFC39F7410
:102E3800019E401F90E40012001EE493FC90064E91
:102E480012001EECF0780A740126F6500418E436D5
:102E5800F650D475F51175D940D2AF22C2AF75D9E5
:102E68000075F522750A00750900AE09AF0A74FFEE
:102E7800C39F74019E401F90D60012001EE493FC6D
:102E880090004E12001EECF0780A740126F65004E9
:102E980018E436F650D4750A00750900AE09AF0A71
:102EA80074FFC39F74019E401F90D80012001EE457
:102EB80093FC90024E12001EECF0780A740126F67C
:102EC800500418E436F650D4750A00750900AE09A6
:102ED800AF0A74FFC39F74019E401F90DA0012006E
:102EE8001EE493FC90044E12001EECF0780A740164
:102EF80026F6500418E436F650D4750A0075090011
:102F0800AE09AF0A74FFC39F74019E401F90DC0096
:102F180012001EE493FC90064E12001EECF0780A94
:102F2800740126F6500418E436F650D475F5117578
:102F3800D940D2AF22E51464046006E59964FF60C5
:102F4800028031A20F4004D20F8027E51460087474
:102F5800E62514900023F0E513600874F02513901B
:102F68000023F0E514B4010280FE75140075130007
:102F7800C20F8002C20FE514903898F8282873759C
:102F88001400E599B4FF03751301E599B4FE0375C0
:102F98001302E599B4FD03751303E599B4FC0375B1
:102FA8001304E599B4FA03751305E599B4FB06759E
:102FB8001401120447E599B4F9067514041204477C
:102FC800E599D394E54007E599C394F0400280164B
:102FD8008599157514027E017F00E515C394E612E4
:102FE8003F6F8E0D8F0E900786E4F0A3F0E599D31E
:102FF80094C44007E599C394E64002802885991552
:1030080075140374E5C39515F50E750D00AE0DAF77
:103018000E9038F512002EE493F874019390078609
:10302800C8F0A3C8F0D2990234AC900786E0FEA39A
:10303800E0FFEFC39400EE94054009EFD394FFEE50
:1030480094064013900786E0FEA3E0FF90004E121E
:10305800001EE599F0800385996C90078612000E92
:10306800900786E0FEA3E0FFEFB40106EEB4070286
:1030780080030232BC90074EE0B43C028003023267
:10308800BCA20AB35005A20BB340030231AFC29CE5
:1030980090007AE090078CF0900057E090078DF050
:1030A800900062E090078EF0900063E090078FF048
:1030B800900074E0900790F090007CE0900791F009
:1030C80090007DE0900792F0900080E0900793F0E8
:1030D800900081E0900794F090013AE0900795F015
:1030E80090013BE0900796F090013CE0900797F044
:1030F800900090E0900798F0900091E0900799F088
:10310800900092E090079AF0900093E090079BF06F
:10311800900094E090079CF0900095E090079DF057
:10312800900096E090079EF0900097E090079FF03F
:10313800900099E09007A0F090009AE09007A1F025
:1031480090009BE09007A2F090009CE09007A3F00D
:103158007400900082F012008F74AB900788F01210
:0A316800263674AA900788F0E55897
:06389800022F870230320E
:103172009038B9F828287380121226E1800D12289F
:0B3182001F800812295D8003122A9BA9
:0F38B90002317902317B02318002318502318A7E
:10318D00900788E4F090013AE0700C90013BE070FC
:10319D000690013CE060028004C20A8002D20A025D
:1031AD0032B1C29C900078E0900789F090005EE00B
:1031BD0090078AF090005FE090078BF090007AE026
:1031CD0090078CF0900057E090078DF0900062E032
:1031DD0090078EF0900063E090078FF0900074E000
:1031ED00900790F090007CE0900791F090007DE0CA
:1031FD00900792F0900080E0900793F0900081E0AE
:10320D00900794F090013AE0900795F090013BE023
:10321D00900796F090013CE0900797F0900090E0B9
:10322D00900798F0900091E0900799F0900092E04F
:10323D0090079AF0900093E090079BF0900094E037
:10324D0090079CF0900095E090079DF0900096E01F
:10325D0090079EF0900097E090079FF0900099E006
:10326D009007A0F090009AE09007A1F090009BE0ED
:10327D009007A2F090009CE09007A3F074009000DE
:10328D0082F074AB900788F012263674AA900788E6
:10329D00F01226E112281F12295D122A9BD29C756D
:1032AD0099FB80FED29C7514007513007599FB0275
:1032BD0034AC900786E0FEA3E0FFEF4E70068599D3
:1032CD0010750F00900786E0FEA3E0FF74016F4EAE
:1032DD00701BAC0FAD10AA0DAB0EED2BFBEC3AFA3B
:1032ED008A068B0790004E12001EE599F090078616
:1032FD0012000E900786E0FEA3E0FF74026F4E7081
:10330D000C12008F8515997514007513000234ACDD
:10331D00900786E0FEA3E0FF90004E12001EE59997
:10332D00F090078612000E900786E0FEA3E0FFAC3A
:10333D000DAD0E8F028E038C068D0790392D120068
:10334D002EE493F9740193FEEAD39EEB994009851F
:10335D0015997514007513000234AC900786E0FEC4
:10336D00A3E0FF90004E12001EE599F09007861223
:10337D00000E900786E0FEA3E0FFEFB40006EEB46A
:10338D00010280030234AC90001CE0D394C7400BC3
:10339D0090001CE0C394C8F516801A90001CE0D371
:1033AD009463400B90001CE0C39464F51680069066
:1033BD00001CE0F516E51675F002A4FFAEF08F6B5C
:1033CD00EF90004E123F87EFFCE0FDEC90005112A4
:1033DD003F87EDFCE0FDEC2DB51602800302349E17
:1033ED000FEF90004E123F87E56BFFE0FCEF900072
:1033FD0052123F87ECFFE0FCEFC39CB51602800331
:10340D0002349EE56B900050123F87E56BFFE0FCA8
:10341D00EF900053123F87ECFFE0FCEF2CB51671D7
:10342D00E56B900054123F87E0C3951690079DF011
:10343D00E56B900055123F87E0C3951690079EF0FF
:10344D00E56B900058123F87E0C3951690079FF0EB
:10345D00E56B900059123F87E0C395169007A0F0D9
:10346D00E56B90005A123F87E0C395169007A1F0C7
:10347D00E56B90005B123F87E0C395169007A2F0B5
:10348D001225AC7599F975186475170012256880A9
:0F349D00FE7599FF75186475170012256880FE7B
:09389E000232BF02331D0233683F
:1034AC0022E5139038A7F82828730235ED9007868B
:1034BC00E0FEA3E0FF90001212001EE0F5999007C9
:1034CC008612000E900786E0FEA3E0FF74116F4E8B
:1034DC0070037513000235ED8562990235ED900786
:1034EC0086E0FEA3E0FF90004E12001EE0F599EF7F
:1034FC00B40107EEB4070375130090078612000E93
:07350C000235ED900787E096
:0F38A7000234B60234B90234E40234EA02350FB7
:103513009038C8F82828738524990235E2852A99BA
:103523000235E28544990235E28547990235E28501
:1035330051990235E28560990235E2855699023543
:10354300E28558990235E2756E00900069E07006D5
:10355300900068E060028016A2A44006E56E440471
:10356300F56EA2A54006E56E4402F56E801A900042
:103573004AE0B40106E56E4410F56E900049E0B4EC
:103583000106E56E4420F56EA207B34006E56E44DE
:1035930001F56EA209B34006E56E4408F56E856E2B
:1035A30099803CA210B340077599FAC2108017A204
:1035B3000CB3400575990F800B900023E0F59990AB
:1035C3000023E4F0C20C80178542998012854B9941
:0F35D300800D85469980087599FC80037513005B
:1038C80002351A02352002352602352C023532021D
:1038D800353802353E02354402354A0235A60235EE
:0D38E800CB0235D00235D50235DA0235DFCE
:0B35E20090078612000E8003120048C4
:0338B6000235EAEE
:1035ED002290006BE0B4010385241190006BE0B4D0
:1035FD000203852A1190006BE0B4030385441190FA
:10360D00006BE0B4040385471190006BE0B4050333
:10361D0085511190006BE0B4060385561190006B37
:10362D00E0B4070385581190006CE0FE90006DE04A
:10363D00C39E50030236C490006BE0D39404402C1B
:10364D0090006CE0D39511500990006DE0C3951179
:10365D0050028002D20090006CE0D3951150099079
:10366D00006DE0C395115002C200804990006BE0DF
:10367D00B4041890006DE0C395115002D200900073
:10368D006CE0D395114002C200802A90006CE0C31B
:10369D009511500990006DE0D3951150028002D222
:1036AD000090006CE0D39511500990006DE0C3952A
:1036BD00115002C200807E90006BE0D39404402C28
:1036CD0090006CE0C39511400990006DE0D3951109
:1036DD0040028002C20090006CE0C3951140099039
:1036ED00006DE0D395114002D200804990006BE04F
:1036FD00B4041890006CE0C395115002C200900004
:10370D006DE0D395114002D200802A90006CE0C389
:10371D009511400990006DE0D395114002D20090B3
:10372D00006CE0D39511400990006DE0C3951140F8
:10373D00028002C2002290006EE0B40103852411C4
:10374D0090006EE0B40203852A1190006EE0B40380
:10375D000385441190006EE0B40403854711900079
:10376D006EE0B4050385511190006EE0B40603853B
:10377D00561190006EE0B4070385581190006FE06C
:10378D00FE900070E0C39E500302381990006EE069
:10379D00D39404402C90006FE0D395115009900004
:1037AD0070E0C3951150028002D20290006FE0D3F9
:1037BD0095115009900070E0C395115002C202801E
:1037CD004990006EE0B40418900070E0C39511505C
:1037DD0002D20290006FE0D395114002C202802AFE
:1037ED0090006FE0C395115009900070E0D39511D2
:1037FD0050028002D20290006FE0D39511500990D3
:10380D000070E0C395115002C202807E90006EE000
:10381D00D39404402C90006FE0C3951140099000A3
:10382D0070E0D3951140028002C20290006FE0C398
:10383D0095114009900070E0D395114002D202809D
:10384D004990006EE0B4041890006FE0C3951150DC
:10385D0002C202900070E0D395114002D202802A7C
:10386D0090006FE0C395114009900070E0D3951161
:10387D004002D20290006FE0D39511400990007084
:0B388D00E0C3951140028002C202223D
:093F87002582F582500205832217
:10002E00EF2F500205832582F582E5833E2EF58360
:01003E00229F
:08000300C3EF9DFFEE9CFE22FD
:08003F000806B60002180622B3
:0D000E00A3E004F07006123F7DE004F02234
:083F99000816B6FF02181622FB
:0E3F6100048007C3CE13CECF13CFD5E0F622D7
:103E0F00BC000FBE0008ED8FF084FFADF022E4FE82
:103E1F00FF22BE000DEF60FE54F0606F20E703023B
:103E2F003EC5EAC0E0EBC0E078017A0075F001EE24
:103E3F0020E710EF25E0FFEE33FE0AC5F023C5F0B3
:103E4F0030E7F0EA5407F9096A7A007B006001084D
:103E5F00C3EC9E40167004ED9F4010ED9FFDEC9E4D
:103E6F00FCE5F0CA4ACA03F5F08005E5F003F5F06A
:103E7F00C3EE13FEEF13FFD9D77908CACBCAD8D038
:103E8F00EAFEEBFFD0E0FBD0E0FA22EC8FF084FCEF
:103E9F00ED54F045F0C48FF084FEEDC454F045F0BE
:103EAF00C48FF084FDEEC4FE54F02DFFEE540F3C92
:103EBF00FEADF07C0022790078008FF0EC7E0820B8
:103ECF00E70DC3CD33CD33C933C9C833C8DEF08452
:103EDF0049F9E5F08FF0BE00E6FD7C00E9FFE8FE52
:013EEF0022B0
:0E3F6F00F88FF0A4FFE5F0CE88F0A42EFE221D
:103F4100600D782B023F4B007830D8FED5E0F82287
:103F5100EEC0E07E00123E0FEFFDEEFCD0E0FE224F
:03000B00023EF0C2
:03001B00023F0B96
:03002B00023F266B
:03000000023F902C
:093F900075817275D0000206274C
:0B001E00E5822FF582E5833EF583228A
:0A3F7D000582D58202158315822209
:103EF000C0E0C0F0C083C082C0D075D00012061CE4
:103F0000D0D0D082D083D0F0D0E032C0E0C0F0C0BA
:103F100083C082C0D075D00012061FD0D0D082D00E
:103F200083D0F0D0E032C0E0C0F0C083C082C0D007
:103F300075D000120622D0D0D082D083D0F0D0E04D
:013F4000324E
:00000001FF
